:100000008A01122820292E29402953295C296E298A
:10001000A529BA29142A202A292A322A422A552A0D
:100020006E2A7C2A02208A110A1207208A110A12DB
:100030003C308312AD0006208A110A120F30831261
:10004000AD0006208A110A1283128701AA0110202E
:100050008A110A120A208A110A128312AB01A50121
:10006000831225080F3C013003190301003C0319DA
:10007000AF288C1E42281A08A6002608AC000420CF
:100080008A110A1209208A110A12103083122502DD
:10009000013003180301003C0319A328AA0801300A
:1000A000031D0301003C0319A22801308312AA009A
:1000B0000A302502013003180301003C031974289B
:1000C000A0012508303E0318A00AAC0004208A11C4
:1000D0000A128312A0012508303E0318A00AB000BE
:1000E00011208A110A1288288312A0012508373EA0
:1000F0000318A00AAC0004208A110A128312A0017E
:100100002508373E0318A00AB00011208A110A12F0
:100110000B208A110A12A0308312AE000D208A1122
:100120000A1283122B08AE000D208A110A128312C4
:100130002508AE000D208A110A120C208A110A121D
:100140008312AB0AA82883122A080319A828AA0137
:100150000A308312A20008208A110A123028C03007
:100160008312AD0006208A110A128312AB010A2005
:100170008A110A120B208A110A12A0308312AE00D3
:100180000D208A110A1283122B08AE000D208A114D
:100190000A120C208A110A120B208A110A12A130AD
:1001A0008312AE000D208A110A128312A501831258
:1001B00025080F3C013003190301003C03191629DF
:1001C0000E208A110A128312A5000A30250201307E
:1001D00003180301003C0319F728A0012508303E4D
:1001E0000318A00AAC0004208A110A120129831204
:1001F000A0012508373E0318A00AAC0004208A118C
:100200000A12831225080F3C0130031D0301003C34
:10021000031910290130AF000F208A110A12152985
:100220008312AF010F208A110A12D7280C208A11DD
:100230000A1202308312AD0006208A110A122D28FC
:1002400083128501F8308316850006309F008312E3
:10025000051005118510831686010800FF308316EE
:100260008600831285148312051100000515000015
:10027000861B3329051100008510831686010800AE
:100280008312851005102C08860003208A110A129B
:10029000831205140515000005112D30A40005205A
:1002A0008A110A120800A40C7F30A4050430A402AD
:1002B000A40B5829000008008312851005102D0892
:1002C000860003208A110A12831205150000051109
:1002D0002D30A40005208A110A1208003C30831238
:1002E000AD0006208A110A1205308312A2000820F0
:1002F0008A110A123C308312AD0006208A110A12BC
:1003000005308312A20008208A110A123C308312A1
:10031000AD0006208A110A1205308312A2000820BF
:100320008A110A1208308312AD0006208A110A12BF
:1003300001308312AD0006208A110A1206308312A2
:10034000AD0006208A110A12080073308312A30040
:10035000000000000000000000000000000000009D
:10036000000000000000A30BA9290000A20BA52992
:1003700000000800F0308316860081138312860186
:100380000609A800A80EA701831228080139FF3921
:100390000130031D0030003C0319D329280C7F399C
:1003A000A800A70AC42904308312270201300318C9
:1003B0000301003C0319102A2708A9000F308316F7
:1003C00086008113831286010609A800A701831203
:1003D00028080139FF390130031D0030003C0319A2
:1003E000F629280C7F39A800A70AE72904308312D0
:1003F0002702013003180301003C03190C2A2708C7
:10040000A800A0012908A100A10D210DFC39280791
:100410000318A00AA5000F2AFF308312A500132A93
:10042000FF308312A50008008316070830388700C4
:10043000803094000E30930028308312940008001E
:1004400083128C11831611148316111C282A242A56
:10045000080083128C11831611158316111D312A81
:100460002D2A080083128C112E08930083120C0889
:100470000839003C0130031D0301003C0319412AE7
:10048000362A080083128C118316911583120C08EA
:100490000839003C0130031D0301003C0319512AB7
:1004A000462A83128C111308080083128C112F081E
:1004B000003C03195E2A83169116602A8316911256
:1004C0008316111683120C080839003C0130031DF5
:1004D0000301003C03196D2A622A080026308316A6
:1004E0009900A43098009030831298008316070872
:1004F000BF3980388700080083123008990008004F
:00000001FF
